S00C0000446F6F722E7372656384
S113000012C017C016C015C014C013C012C011C04E
S113001010C00FC00EC00DC00CC00BC00AC009C078
S113002008C007C006C011241FBECFEDCDBF11D03C
S113003035C0E6CF18B883E081B90895BA9A8D9A8D
S1130040089581EB80BF81E083BF12BE16BE1CBE43
S11300500895F0DFF3DFF5DF459B10C086B78823F2
S1130060D9F386B7815086BF8CB781508CBF8FEC93
S113007097E00197F1F700C00000EECF86B78F3FFD
S113008059F386B78F5F86BF8CB78F5F8CBF8FEDB8
S11300909EE20197F1F700C00000DECFF894FFCF95
S9030000FC
